:020000040000FA
:1000000025006300D50C0200080C0600670069009B
:1000100001030F0EC9011809260001070D0A010688
:100020000F0A21024307080AA9023F0C6901080AC6
:100030003F0EE2010E080E080E080E080E080E080C
:100040000E080E080E080E080E080E080E080E0800
:100050000E080E080D080D080D080D080D080D08F6
:100060000D080D080D080D080D080D080D080D08E8
:100070000D080D080B080B080B080B080B080B08E4
:100080000B080B080B080B080B080B080B080B08D8
:100090000B080B080D080D080D080D080D080D08BC
:1000A0000D080D080D080D080D080D080D080D08A8
:0400B0000D080D0822
:0203FE00240CCD
:021FFE001800C9
:00000001FF
